:1000000012C02CC02BC02AC029C028C027C026C0BF
:1000100025C024C023C06EC021C020C01FC01EC088
:100020001DC01CC01BC011241FBECFE5D4E0DEBF25
:10003000CDBF11E0A0E6B0E0EEE0F2E002C0059036
:100040000D92A438B107D9F712E0A4E8B1E001C0DD
:100050001D92A530B107E1F741D0D8C0D1CF8A9A1F
:10006000929AB89AC09810BC87E189B988E98AB990
:1000700078940895AC0183E083BF20E030E009C0AC
:1000800081E088BF86EC82BF08B600FEFDCF2F5FFF
:100090003F4F24173507A1F708955D9BFECF8CB91C
:1000A0000895FC0104C05D9BFECF8CB93196808120
:1000B0008823C9F7089580E690E0F3DF8DE890E0AB
:1000C000F0DF87EB90E0EDDF8DEC90E0EADF8FEE84
:1000D00090E0E7DF80E191E0E4DF0895CFE5D4E050
:1000E000DEBFCDBFBCDF929888EB9BE0C3DF929A66
:1000F000E2DFFFCF1F920F920FB60F9211242F93C2
:100100003F934F935F936F937F938F939F93AF939F
:10011000BF93EF93FF939CB1892F81568A3108F4E6
:100120009052809104028F3758F4903248F0E82FB3
:10013000FF27EC57FE4F90838F5F8093040240C0EF
:100140009A30F1F545E050E060E371E084E891E039
:100150004FD0892B51F486E391E0A3DFC09A9298A7
:1001600088EE93E087DFC098929A47E050E063E51D
:1001700071E084E891E03CD0892B51F48BE591E06B
:1001800090DFC09A929880E197E274DFC098929ACB
:1001900044E050E06EE771E084E891E029D0892BDB
:1001A00031F489DF929888EC90E064DF929A40E81D
:1001B00050E060E270E084E891E013D01092040215
:1001C000FF91EF91BF91AF919F918F917F916F912F
:1001D0005F914F913F912F910F900FBE0F901F9005
:1001E0001895DC0101C06D9341505040E0F708952F
:1001F000FB01DC014150504030F08D91019080199D
:0E02000019F40020B9F7881B990B0895FFCF61
:10020E000D0A0A415652204D6567613820617320F0
:10021E005752543534474C206164642D6F6E2069FB
:10022E007320616C6976652E2E2E0D0A00286329C7
:10023E0020323030382062792048657262657274DF
:10024E002044696E6766656C6465722C20444C357B
:10025E004E45470D0A0A00417661696C61626C6514
:10026E0020636F6D6D616E64733A0D0A00415450D8
:10027E004342202020537461727473207468652089
:10028E00636F6E6E65637465642050430D0A0041A2
:10029E005450434F464620466F7263657320746810
:1002AE00652050432068617264206F66660D0A00F7
:1002BE0048454C502020202053686F777320746877
:1002CE0069732068656C7020746578740D0A0A0075
:1002DE00415450434200504320626F6F7420636F4D
:1002EE006D6D616E6420726563656976656421204B
:1002FE000D0A00415450434F464600504320666F4E
:10030E0072636564206F666620636F6D6D616E64E7
:10031E0020726563656976656421200D0A00484583
:04032E004C5000002F
:00000001FF
